:0A0026001217DB1218B51214C322E2
:0300330002001DAB
:04001D0053D8EF3293
:100006008E128F13E5131513AE12700215124E6081
:07001600051218A480EE2280
:03000300020046B2
:10004600C0E0C083C082C086758600C0D075D00867
:1000560030990E301107A217929B854699C299D204
:100066001F30C10E301207A21892C38547C1C2C104
:10007600D220201F03020442C21F2003030202678C
:10008600201103020138E54AC3957C503E20133601
:10009600200B33907F9BE020E303201C29301B12AA
:1000A600AE4A054A74402EF582E4347EF583E013A9
:1000B6009217AE4A054A74402EF582E4347EF583E3
:1000C600E0F546020440C211020440907FC7E4F006
:1000D600C20330150CC215907FBF04F0C211020492
:1000E60040907FC8E030E105C211020440907FC90C
:1000F600E0F57C907DC0E013921520132D200B2A8D
:03004300021B009D
:0300230002004692
:03003B000200467A
:0300000002163DA8
:40010600907F9BE020E303201C20301B11907DC1E0139217A3E0F546754A03020440754A02907DC1E0F546020440754A01C211020440E54AC3957C50030201E0907FC6E08A
:4001460030E107C221C205020440907FC7E0F57C907E40E01392153013030201D8200B7220006F907F9BE020E303201C65301B10907E41E013929BA3E0F599754A038009BE
:40018600907E41E0F599754A02E54AC3957C4017907FC7E4F0C203201503020440C215907FBF04F0020440301B12AE4A054A74402EF582E4347EF583E0139217AE4A054AA7
:4001C60074402EF582E4347EF583E0F546D211020440754A01C221020440301303020262200B79907F9BE020E303201C6F301B12AE4A054A74402EF582E4347EF583E013DC
:40020600929BAE4A054A74402EF582E4347EF583E0F599E54AC3957C4017907FC7E4F0C203201503020440C215907FBF04F0020440301B12AE4A054A74402EF582E4347EB6
:40024600F583E0139217AE4A054A74402EF582E4347EF583E0F546D211020440C221020440201103020319E54AC3957C503E201336200B33907F9BE020E303201C29301B5F
:4002860012AE4A054A74C02EF582E4347DF583E0139217AE4A054A74C02EF582E4347DF583E0F546020440C211020440907FC9E4F0D20330150CC215907FBF04F0C2110276
:4002C6000440907FC6E030E105C211020440907FC7E0F57C907E40E013921520132D200B2A907F9BE020E303201C20301B11907E41E0139217A3E0F546754A03020440759E
:400306004A02907E41E0F546020440754A01C211020440E54AC3957C50030203C1907FC8E030E107C221C205020440907FC9E0F57C907DC0E01392153013030203B9200B48
:400346007220006F907F9BE020E303201C65301B10907DC1E013929BA3E0F599754A038009907DC1E0F599754A02E54AC3957C4017907FC9E4F0D203201503020440C21573
:40038600907FBF04F0020440301B12AE4A054A74C02EF582E4347DF583E0139217AE4A054A74C02EF582E4347DF583E0F546D211020440754A01C221020440301303020463
:4003C6003E200B74907F9BE020E303201C6A301B12AE4A054A74C02EF582E4347DF583E013929BAE4A054A74C02EF582E4347DF583E0F599E54AC3957C4013907FC9E4F09D
:40040600D203301535C215907FBF04F0802C301B12AE4A054A74C02EF582E4347DF583E0139217AE4A054A74C02EF582E4347DF583E0F546D2118002C221D2252020030230
:40044600080CC220200403020631201203020502E54BC3957D503E201436200D33907F9AE020E503201E29301D12AE4B054B74402EF582E4347DF583E0139218AE4B054B99
:4004860074402EF582E4347DF583E0F54702080AC21202080A907FCBE4F0C20430160CC216907FC104F0C21202080A907FCCE030E105C21202080A907FCDE0F57D907CC0BB
:4004C600E013921620142D200D2A907F9AE020E503201E20301D11907CC1E0139218A3E0F547754B0302080A754B02907CC1E0F54702080A754B01C21202080AE54BC39566
:400506007D50030205AA907FCAE030E107C222C20602080A907FCBE0F57D907D40E01392163014030205A2200D7220006F907F9AE020E503201E65301D10907D41E013920D
:40054600C3A3E0F5C1754B038009907D41E0F5C1754B02E54BC3957D4017907FCBE4F0C20420160302080AC216907FC104F002080A301D12AE4B054B74402EF582E4347D24
:40058600F583E0139218AE4B054B74402EF582E4347DF583E0F547D21202080A754B01C22202080A30140302062C200D79907F9AE020E503201E6F301D12AE4B054B7440E9
:4005C6002EF582E4347DF583E01392C3AE4B054B74402EF582E4347DF583E0F5C1E54BC3957D4017907FCBE4F0C20420160302080AC216907FC104F002080A301D12AE4B91
:40060600054B74402EF582E4347DF583E0139218AE4B054B74402EF582E4347DF583E0F547D21202080AC22202080A2012030206E3E54BC3957D503E201436200D33907F1A
:400646009AE020E503201E29301D12AE4B054B74C02EF582E4347CF583E0139218AE4B054B74C02EF582E4347CF583E0F54702080AC21202080A907FCDE4F0D20430160C43
:40068600C216907FC104F0C21202080A907FCAE030E105C21202080A907FCBE0F57D907D40E013921620142D200D2A907F9AE020E503201E20301D11907D41E0139218A352
:4006C600E0F547754B0302080A754B02907D41E0F54702080A754B01C21202080AE54BC3957D500302078B907FCCE030E107C222C20602080A907FCDE0F57D907CC0E013AC
:400706009216301403020783200D7220006F907F9AE020E503201E65301D10907CC1E01392C3A3E0F5C1754B038009907CC1E0F5C1754B02E54BC3957D4017907FCDE4F0AE
:40074600D20420160302080AC216907FC104F002080A301D12AE4B054B74C02EF582E4347CF583E0139218AE4B054B74C02EF582E4347CF583E0F547D21202080A754B0173
:40078600C22202080A301403020808200D74907F9AE020E503201E6A301D12AE4B054B74C02EF582E4347CF583E01392C3AE4B054B74C02EF582E4347CF583E0F5C1E54B3F
:4007C600C3957D4013907FCDE4F0D204301635C216907FC104F0802C301D12AE4B054B74C02EF582E4347CF583E0139218AE4B054B74C02EF582E4347CF583E0F547D2122A
:400806008002C222D22520980302093EC2982001030208B0202327AE48054874802EF582E4347EF583E599F0301B49AE48054874802EF582E4347EF583E598F08036AF996E
:40084600EFB55804D20B802CEFB55704C20B8024AE48054874802EF582E4347EF583EFF0301B11AE48054874802EF582E4347EF583E598F0D219E548C39554500302093C9F
:40088600907FB8E030E115E548C39440500302093C15481548052DD20C02093C907FB7E548F0754800C20102093C202327AE48054874002EF582E4347EF583E599F0301BBF
:4008C60049AE48054874002EF582E4347EF583E598F08036AF99EFB55804D20B802CEFB55704C20B8024AE48054874002EF582E4347EF583EFF0301B11AE48054874002E51
:40090600F582E4347EF583E598F0D219E548C395544023907FB6E030E111E548C39440401515481548052DD20C800B907FB9E548F0754800D201D22520C003020A70C2C016
:400946002002030209E2202427AE49054974802EF582E4347DF583E5C1F0301D49AE49054974802EF582E4347DF583E5C0F08036AFC1EFB57004D20D802CEFB56F04C20DAE
:400986008024AE49054974802EF582E4347DF583EFF0301D11AE49054974802EF582E4347DF583E5C0F0D21AE549C3956C5003020A6E907FBCE030E115E549C39440500351
:4009C600020A6E154915490539D20E020A6E907FBBE549F0754900C202020A6E202427AE49054974002EF582E4347DF583E5C1F0301D49AE49054974002EF582E4347DF555
:400A060083E5C0F08036AFC1EFB57004D20D802CEFB56F04C20D8024AE49054974002EF582E4347DF583EFF0301D11AE49054974002EF582E4347DF583E5C0F0D21AE54983
:400A4600C3956C4023907FBAE030E111E549C394404015154915490539D20E800B907FBDE549F0754900D202D225302505C225020056D0D0D086D082D083D0E032907FCE99
:400A8600E030E103020BA5E4F51274402512F582E4347CF583E0FFE5127C007B00244CF9EC3400FAEF1215CD0512E512B418DBE54C600C75C92075C836854DCA854ECBE5BC
:400AC6004F13921B929FE55013921CE551139223E5526009907F98E054FBF08007907F98E04404F0E5536009907F98E0547FF08007907F98E04480F0E559600BC213C20B18
:400B0600907F95E04402F0E55A600BD20BD20C907F95E04402F0E55B600DC2AFC211D200E4F57CF54AD2AFE55C6005302302D20BE55D6015907F95E054FDF0907F9EE044D9
:400B460002F0907F98E054FDF0E55E600AD29CC298752E01754028E55F6007C29CE4F548F52EE5606003E4F548E5616002D207E5626008E55E7002F540D20CE56360199060
:400B86007FD77411F07431F07412F07432F07415F07435F0D203D201D209E4907FCFF0A213E433FF652B60048F2BD20CA20BE433FF652C60048F2CD20C907F9BE054086589
:400BC600276007E05408F527D20C907F9BE05440B52909E054406440F529D20C300735C2AF300118907FB8E020E127E5486009907FB7F0E4F548C201C2078016907FB6E0E9
:400C060020E10FE5486009907FB9F0E4F548D201C207D2AF20053730031B907FC6E020E12D907E40E0139215754A01907FC7E0F57CD2058019907FC8E020E112907DC0E0CF
:400C4600139215754A01907FC9E0F57CD205202133200006E54A657C702A30051A300309E4907FC7F0C2038007E4907FC9F0D203C205E4F57CF54A30150AC215C200907F5C
:400C8600BF7401F0302103020D94200503020D94301C0A907F9BE020E303020D94300B03020D94301303020D94300362301B12AF4A054A74402FF582E4347EF583E01392CE
:400CC6002DAF4A054A74402FF582E4347EF583E0F513E54AC3957C502A301B12AF4A054A74402FF582E4347EF583E0139217AF4A054A74402FF582E4347EF583E0F546D266
:400D060011806BC211E4907FC7F0C2038060301B12AF4A054A74C02FF582E4347DF583E013922DAF4A054A74C02FF582E4347DF583E0F513E54AC3957C502A301B12AF4A67
:400D4600054A74C02FF582E4347DF583E0139217AF4A054A74C02FF582E4347DF583E0F546D2118009C211E4907FC9F0D203301B04A22D929BD221C2AF85139920110D3043
:400D8600150AC215C200907FBF7401F0D2AF907FD0E030E103020EB5E4F51274C02512F582E4347BF583E0FFE5127C007B002464F9EC3400FAEF1215CD0512E512B418DB51
:400DC600E564600B758960758840D2DF85658DE56713921D92C7E56813921EE569139224E56A6009907F97E054EFF08007907F97E04410F0E56B6009907F97E0547FF080A4
:400E060007907F97E04480F0E571600BC214C20D907F94E04408F0E572600BD20DD20E907F94E04408F0E573600DC2AFC212D200E4F57DF54BD2AFE5746005302402D20D20
:400E4600E5756015907F94E054F7F0907F9DE04408F0907F97E054F7F0E576600AD2C4C2C0753A01754128E5776007C2C4E4F549F53AE5786003E4F549E5796002D208E5F0
:400E86007A6008E5767002F541D20EE57B6019907FD77413F07433F07414F07434F07416F07436F0D204D202D20AE4907FD1F0A214E433FF653760048F37D20EA20DE43304
:400EC600FF653860048F38D20E907F9AE0542065336007E05420F533D20E907F9AE05440B53509E054406440F535D20E300835C2AF300218907FBCE020E127E54960099099
:400F06007FBBF0E4F549C202C2088016907FBAE020E10FE5496009907FBDF0E4F549D202C208D2AF20063730041B907FCAE020E12D907D40E0139216754B01907FCBE0F503
:400F46007DD2068019907FCCE020E112907CC0E0139216754B01907FCDE0F57DD206202233200006E54B657D702A30061A300409E4907FCBF0C2048007E4907FCDF0D2042C
:400F8600C206E4F57DF54B30160AC216C200907FC17401F03022030210A42006030210A4301E0A907F9AE020E5030210A4300D030210A43014030210A4300462301D12AF8E
:400FC6004B054B74402FF582E4347DF583E013922DAF4B054B74402FF582E4347DF583E0F513E54BC3957D502A301D12AF4B054B74402FF582E4347DF583E0139218AF4B78
:40100600054B74402FF582E4347DF583E0F547D212806BC212E4907FCBF0C2048060301D12AF4B054B74C02FF582E4347CF583E013922DAF4B054B74C02FF582E4347CF5F2
:4010460083E0F513E54BC3957D502A301D12AF4B054B74C02FF582E4347CF583E0139218AF4B054B74C02FF582E4347CF583E0F547D2128009C212E4907FCDF0D204301DF4
:4010860004A22D92C3D222C2AF8513C120120D30160AC216C200907FC17401F0D2AF907FC2E030E10302117AE51A7046300C3FE540703BA20933F531C209C20CE4F5127E0D
:4010C600007B0074262512F9EE3400FA121587FF74802512F582E4347BF583EFF00512E512B40CDB907FC3740CF075401022751A0122E51A64017045300E3EE541703AA2C5
:401106000A33F53DC20AC20EE4F5127E007B0074322512F9EE3400FA121587FF74802512F582E4347BF583EFF00512E512B40CDB907FC3740CF0754110751A0222E51C60CA
:4011460030151CE4F5127E007B00741B2512F9EE3400FA121587FF74802512F582E4347BF583EFF00512E512B403DB907FC37403F0E4F51A22907FE9E012161712400012A7
:40118600B401132003119E06123308122D0912200A13760B0000136F907FEBE024FE6016146040240270697419907FD4F07400907FD5F0021376907FEAE0FF12174B8B1261
:4011C6008A138914EA496011AE02EE907FD4F0AF01EF907FD5F0021376907FB4E04401F0021376907FEAE0FF12179A8B128A138914EA496011AE02EE907FD4F0AF01EF9083
:401206007FD5F0021376907FB4E04401F0021376907FB4E04401F0021376907F007401F0907FB5F00213761214C3021376907F007401F0907FB5F0021376907FE8E0247FBF
:4012460060241460312402705BA226E433FF25E0FFA22BE4334F907F00F0E4A3F0907FB57402F0021376E4907F00F0A3F0907FB57402F0021376907FECE0F45480FFC45429
:401286000FFFE054072F25E024B4F582E4347FF583E054FD907F00F0E4A3F0907FB57402F0021376907FB4E04401F0021376907FE8E024FE601D24026003021376907FEA0B
:4012C600E0B40105C226021376907FB4E04401F0021376907FEAE07038907FECE0F45480FFC4540FFFE054072F25E024B4F582E4347FF583E4F0907FECE05480FF131313A7
:40130600541FFFE054072F907FD7F0E04420F0805F907FB4E04401F08056907FE8E024FE60182402704A907FEAE0B40104D226803F907FB4E04401F08036907FEAE07020A3
:40134600907FECE0F45480FFC4540FFFE054072F25E024B4F582E4347FF5837401F08010907FB4E04401F08007907FB4E04401F0907FB4E04402F0222028030214C2E54063
:4013860060021540E548604F65447045E542F460020542E542C39555403DC2AF300118907FB8E020E127907FB7E548F0C201E4F548F542F5448016907FB6E020E10F907F07
:4013C600B9E548F0D201E4F548F542F544D2AF8006854844E4F542E52E602D201907907F9BE030E00EE52F6005E4F52FD20CE4F53E8013E53ED39556500CE53EB556057504
:401406002F01D20C053EC219E54160021541E549604F65457045E543F460020543E543C3956D403DC2AF300218907FBCE020E127907FBBE549F0C202E4F549F543F54580E2
:4014460016907FBAE020E10F907FBDE549F0D202E4F549F543F545D2AF8006854945E4F543E53A602D201A07907F9AE030E20EE53B6005E4F53BD20EE4F53F8013E53FD35E
:40148600956E500CE53FB56E05753B01D20E053FC21A907FD2E020E123907B40E06009E0F51C907B42E0F51D907B41E06009907FD77417F07437F0E4907FD3F022E4907FC5
:4014C60093F0907F9C7430F0907F96E04410F0907F94740DF0907F9D749AF0907F97E054FDF0907F957423F0907F9E7484F0E4907FC7F0907FC9F0907FCFF075984043A89E
:4015060010C21BC205C221C20BC213F57CF54AC211C215F542C219F544F548C223C21CF52DF52FC207C200C21FF53EC209D20CF526907FCBF0907FCDF0907FD1F075C04043
:4015460043A840C21DC206C222C20DC214F57DF54BC212C216F543C21AF545F549C224C21EF539F53BC208C200C220F53FC20AD20E753201907FDF74FFF0907FDEF0D228DE
:4015860022BB010689828A83E0225002E722BBFE02E32289828A83E49322BB010CE58229F582E5833AF583E0225006E92582F8E622BBFE06E92582F8E222E58229F582E553
:4015C600833AF583E49322BB010689828A83F0225002F722BBFE01F322BB0110E58229F582E5833AF583E0F5F0A3E0225009E92582F886F008E622BBFE0AE92582F8E2F511
:40160600F008E222E5832AF583E993F5F0A3E99322D083D082F8E4937012740193700DA3A393F8740193F5828883E4737402936860EFA3A3A380DF787FE4F6D8FD75817D0E
:401646000216840216C9E493A3F8E493A34003F68001F208DFF48029E493A3F85407240CC8C333C4540F4420C8834004F456800146F6DFE4800B010204081020408090181A
:40168600C5E47E019360BCA3FF543F30E509541FFEE493A360010ECF54C025E060A840B8E493A3FAE493A3F8E493A3C8C582C8CAC583CAF0A3C8C582C8CAC583CADFE9DE39
:4016C600E780BE751101907F92E054FDF0907FAEE0FFD39226E433FEEF4EF0D2E843D820907FDE7401F0907FDFF0907FAB74FFF0907FA9F0907FAAF05391EF907FAFE044C5
:4017060001F0907FAEE0440DF0D2AFD2BCD2BED22D12187FC227C225C228302803120A83907FD8E065106008E0F51012137E80EA302707C22712117B80E0302CDDC22C12C5
:40174600002680D622E4FE7517FF751819751912AB17AA18A9199000011215A06402702DAD060EEDB50701229000021215DF85F015F5166215E5156216E516621529FDE551
:40178600153AA9057517FFF518891980C37B007A007900228F15E4F5167517FF751819751986AB17AA18A9199000011215A0B4031DAF160516EFB51501221215877E0029BE
:4017C600FFEE3AA9077517FFF518891980D47B007A00790022E4907F93F0907F9CF0907F94F0907F9D7402F0907F97F0E4907F95F0907F9E74FFF0E4907F98F0907F9DF003
:4018060022C0E0C083C082C085C084C086758600907FC4E4F05391EF907FAB7404F0D086D084D085D082D083D0E032C0E0C083C082C085C084C086758600D2275391EF9024
:401846007FAB7401F0D086D084D085D082D083D0E032C0E0C083C082C085C084C086758600D22C5391EF907FAB7408F0D086D084D085D082D083D0E032907FD6E054FBF0DD
:40188600E04408F0302D04E04402F07FF47E01120006907FD6E054F7F0E04404F0227400F58690FDA57C05A3E582458370F922907FD6E04480F0438701000000000022C125
:4018C600AA011A00031B030000C127C12CC126C12B000000000000000000000000000000000000000000000000000000000000000000000000000000000012011001FF0031
:401906000040CD060F0100000102000109027400010100A032090400000EFF0000000705010240000007050202400000070503024000000705040240000007050502400078
:4019460000070506024000000705070240000007058102400001070582024000010705830240000107058402400001070585024000010705860240000107058702400001F3
:401986000403090448034B00650079007300700061006E002C002000610020006400690076006900730069006F006E0020006F006600200049006E006E006F005300790040
:4019C6007300200049006E0063002E0036034B00650079007300700061006E0020005500530042002000530065007200690061006C002000410064006100700074006500F9
:401A0600720000000000000000000000000000000000000000000000000000000000000000000000000000000000000000000000000000000000000000000000000000002E
:401A46000000000000000000000000000000000000000000000000000000000000000000000000000000000000000000000000000000000000000000000000000000000060
:401A86000000000000000000000000000000000000000000000000000000000000000000000000000000000000000000000000000000000000000000000000000000000020
:401AC6000000000000000000000000000000000000000000000000000000000000000000000000000000000000000000000000000000000000000000000002183100021B78
:091B06000400021807000218583F
:00000001FF
